:10000000830100308A0004288301DF298312BD00A8
:10001000BE1B11283E088A003D08BD0A0319BE0A0E
:10002000820083133E1883173D08BD0A8400000830
:1000300008000C3448344F344F3444344D34493480
:10004000433452344F342034533465347234693479
:1000500061346C3420344234693474346234613431
:100060006E34673420344534783461346D34703400
:100070006C34653400340A340D34253464343A3435
:1000800020342534633400340A340D3443346F345F
:100090007034793472346934673468347434203499
:1000A0002834633429342034323430343034353415
:1000B0002C3420344B343934733470347534643414
:0A00C00020344C344C344334003437
:1002E60000300B2AB6000030371836070310B60D5B
:1002F6000310B70CB708031908007729BA01BB0128
:100306000310B90CB80C031C8F293608BA07370836
:100316000318370ABB070310B60DB70D38083904A2
:10032600031900348329051C9629AA21051C962940
:10033600F830A700AA21AC210310051C0314A60C53
:10034600A821A70F9E29260808000000AF29000053
:10035600AE29AD29AE29AF29B029B129B229B329D1
:10036600B429B529B6290800B400F730B5008B13B7
:10037600050804388500D521D321B50A0319CC29EF
:10038600B40C031CBC29FB3900008500D321D621FF
:10039600C029CD29FB3985008B17D521D521080029
:1003A6000000D729D629D729D829D929DA29DB293E
:1003B600DC29DD29DE2908008312A1018B018501D4
:1003C60007309900EB30831685008312FF238316CE
:1003D600900019308312A7000030A8007321443022
:1003E600A7000030A800732105169621A00005126B
:0A03F6003B30A7000030A8002008EB
:10040000A400A501A10A2108A200A3012230A60090
:100410007321F72904288312AF00AD012608AA0032
:10042000B22B2E08253A031DA52BFF30AB00AC01E3
:10043000A9016F2BAF080319202A2F08840080011F
:100440002D0808000230AA072A0284000008A32B06
:10045000A90A2E2A0830AB07FE30AB070230AA07E4
:100460002A0284000008B000840A0008B10029189C
:10047000B11F412AB009B109B00A0319B10AAC038E
:10048000422AA9010B30AB072B08B800B90131088B
:10049000B7003008B600C5233608AE002B08B800F8
:1004A000B9013008B6003108B700C5233A08B000DA
:1004B0003B08B100B201B20AB30133083102031D97
:1004C000632A32083002031C802A2B08B800B901C5
:1004D0003208B6003308B70081213A08B2003B0861
:1004E000B300AC035D2AAD0AAF0803197D2A2F08BB
:1004F000840020308000AF0A802A20308312B72188
:10050000AC032C08803A7F3E0318732A291C932AD7
:10051000AD0AAF080319902A2F0884002D30C32A92
:100520002D308312B7212B08B800B9013208B6006C
:100530003308B700C5233A08B2003B08B3003204C1
:100540000319C92A3308B9003208B8003108B700C6
:100550003008B600C5233A08B6003B08B7002B08A0
:10056000B800B901C5233608AC00803A763E031CBA
:10057000BB2A0730AC07AD0AAF080319C62A2F08FB
:1005800084002C08303E8000AF0A932A2C08303EAD
:10059000912A0A302E02031CCF2A0730AE07AD0A7B
:1005A000AF080319D82A2F0884002E08303EAC2B40
:1005B0002E08303EB02BAD0AAF080319E52A2F08EC
:1005C000840020308000AF0AE82A20308312B7214F
:1005D000AC032C08803A7E3E0318DB2A0230AA07BF
:1005E0002A0284000008AE00A52B0230AA072A02C6
:1005F00084000008B200840A0008B300AE012E088F
:100600003207BD003308BE003D080318BE0A0620AD
:10061000003803190D2BAE0AFF2A2B082E020318EF
:10062000132B2E08AB002B08AC1B3E2BFF3A2C07DC
:10063000031C3E2BAD0AAF080319242B2F0884009E
:1006400020308000AF0A272B20308312B721AC0363
:10065000132B3308BE0032080620AE00B20A03197D
:10066000B30AAD0AAF0803193B2B2F0884002E08EC
:100670008000AF0A3E2B2E088312B721AB032B0F4D
:10068000292BB22B2808BE00270806202A3A031D72
:100690004F2B0230AA072A02840000086B2B28087F
:1006A000BE0027080620D03EAB00A70A0319A80AFF
:1006B0002808BE0027080620AE0030302E02031C9A
:1006C0006F2B3A302E0203186F2B0A30B7002B081D
:1006D00075212E07D03EAB00A70A0319A80A2808E7
:1006E000BE002708A70A0319A80A0620AE00003A90
:1006F00003191A2A2A3A0319222A043A0319422B07
:10070000763A03192A2A3B3A0319E92A073A0319C8
:10071000282A0B3A03192C2A1C3A0319F52A063AFF
:1007200003192E2A0D3A03192A2A30302E02031CEF
:10073000A52B3A302E020318A52B0A30B7002C083F
:1007400075212E07D03EAC006F2BAD0AAF08031900
:10075000AF2B2F0884002E088000AF0AB22B2E0882
:100760008312B7212808BE002708A70A0319A80A80
:100770000620AE00AE08031D112AAF080319C32BD3
:100780002F08840080012D080800BC01BA01BB01BC
:1007900038083904031DCF2BB601B70100341F30D0
:1007A000BC040310BC0AB80DB90D031CD22BB90C44
:1007B000B80C39083702031DDF2B38083602031C3A
:1007C000E72B3808B6023908031C390AB702BA0DFC
:1007D000BB0DBC0BBC1AD72BBC1FF32BBA09BA0A32
:1007E0000319BB03BB093A08B8003B08B9003C1F1A
:0E07F0000034B609B60A0319B703B70900347E
:02400E00E43F8D
:00000001FF
